:1000000009C016C015C014C013C012C011C010C062
:1000100065C00EC011241FBECFE9CDBF20E0A0E611
:10002000B0E001C01D92A736B207E1F77CD05BC1FA
:10003000E7CF87B18074836087B9369A3699FECF4F
:1000400084B125B190E0922B0895EBE2F1E0319775
:10005000F1F700C000000197C1F70895EF92FF92F9
:100060001F93CF93DF931F92CDB7DD27162FE82E76
:10007000F12CC701798323D16981681711F0C70179
:1000800025D18FEFE81AF80AC70119D1181749F0DE
:10009000612FC7010F90DF91CF911F91FF90EF90DB
:1000A00015C10F90DF91CF911F91FF90EF900895B0
:1000B0000F931F93CF93082F10E0C80100D1C82FD2
:1000C000C8010196FCD02C2F30E0322F2227A90145
:1000D000482BCA01CF911F910F9108951F920F9243
:1000E0000FB60F9211248F939F93AF93BF9380917C
:1000F000600090916100A0916200B0916300019650
:10010000A11DB11D8093600090936100A0936200D7
:10011000B0936300BF91AF919F918F910F900FBEED
:100120000F901F90189583B7826083BF8FB583604F
:100130008FBDF894A89580E481BD789417B886B1F6
:10014000826886B9BA9AB99AB89ABB988FB58F77F0
:100150008FBDC09A84EF91E078DF8FB58F778FBD28
:10016000C09884E690E071DF8FB58F7D8FBDC19A16
:1001700084EF91E06ADF8FB58F7D8FBDC19884E6F3
:1001800090E063DFC29A84EF91E05FDFC29884E67B
:1001900090E05BDF109264004CDF909366008093E8
:1001A000650060E070E084E059DF94E0E92EBB2454
:1001B000B39422E0A22E34E6F32EC12CD12C39DFE9
:1001C000EC0180916500909166008C179D0720F0EE
:1001D0008C010C1B1D0B03C08E01081B190B809199
:1001E0006400843029F4C29A84EF91E02EDFC29833
:1001F000C601800F911F6C01D694C79484EF91E0E3
:1002000024DF2BE0C216D104D0F2D0936600C09355
:10021000650080E04DDFC817D90718F4BE0180E003
:100220001DDFC23B82E0D80718F0A092640012C024
:10023000CE01885691408A34914018F4B0926400FF
:1002400009C0CC52D140EC9718F41092640002C05F
:10025000E0926400C2988FB58F778FBDC0988FB53C
:100260008F7D8FBDC198809164008130D9F050F0AE
:100270008230E9F08430F9F4C29A84EF91E0E5DE4F
:10028000C29819C08FB580688FBDF6BE84E010DFBC
:1002900060916500709166006817790760F484E0EA
:1002A000DDDE09C08FB580628FBDF9BC04C08FB59B
:1002B00080688FBDF6BE84EF91E0C7DE7ECFE19906
:1002C000FECF8EBBE09A99278DB30895262FE19932
:1002D000FECF1CBA8EBB2DBB0FB6F894E29AE19A02
:0A02E0000FBE01960895F894FFCFB9
:00000001FF
